:020000020000FC
:100000007ACF18951895189528CE8FC918951895F8
:10001000F8CC1895189518951895189500C6189548
:100020001895000000000000000E111B1115110EA4
:100030000E1F151F1F1B0E0A1B1F1F0E0E04040E82
:100040001F1F0E04000E04151F150404040E0E1FBE
:100050001F040E0000040E0400001F1F1B111B1FB5
:100060001F00040A110A04001F1B1111111B1F039A
:1000700003040E11110E0E11110E040E04060505D7
:10008000040418180C0A0909091B1B00040E1B0E96
:100090000400080C0E0F0E0C0802060E1E0E0602BF
:1000A000040E0404040E040A0A0A0A0A000A1F1DA8
:1000B0001D050505050F100E110E011E0000001F85
:1000C0001F0000040E040E04000E040E04040404B9
:1000D0000404040404040E040000021F02000000D3
:1000E00000081F0800000000101010101F00000A78
:1000F0001F0A00000000040E1F00000000001F0E79
:1001000004000000000000000004040404040004D3
:100110000A0A0A000000000A0A1F0A1F0A0A040F3E
:10012000140E051E041819020408130308141409F8
:1001300015120D060204000000000204080808045D
:10014000020804020202040804150E040E1504003D
:1001500004041F0404000000000006020400000064
:100160001F00000000000000000606000102040855
:1001700010000E11111111110E040C040404040ED0
:100180000E11010204081F1F02040201110E0206D3
:100190000A121F02021F101E0101110E0E11101E65
:1001A00011110E1F0102020404040E11110E11118F
:1001B0000E0E11110F01110E000C0C000C0C0000A2
:1001C0000C0C000C04080204081008040200001FB4
:1001D000001F0000080402010204080E11010204BD
:1001E00000040E11171517100E040A11111F11111A
:1001F0001E11111E11111E0E11101010110E1C12C5
:10020000111111121C1F10101E10101F1F10101E94
:100210001010100E11101711110F1111111F1111C3
:10022000110E04040404040E0F02020202120C1147
:100230001214181412111010101010101F111B1589
:1002400015151111111119151311110E111111118B
:10025000110E1E11111E1010100E11111115120D7C
:100260001E11111E1412110E11100E01110E1F0479
:1002700004040404041111111111110E11111111B2
:10028000110A041111111515150A11110A040A1188
:100290001111110A040404041F01020408101F0EA6
:1002A00008080808080E001008040201000E0202E7
:1002B0000202020E040A110000000000000000000B
:1002C000001F0C08040000000000000E010F110FB9
:1002D00010101E1111111E00000F1010100F01013F
:1002E0000F1111110F00000E111F100E0304041F37
:1002F00004040400000F110F010E10101619111143
:100300001104000C0404040E0200060202120C0088
:100310001012141814120C04040404040E00000A31
:10032000151511110000161911111100000E1111EF
:10033000110E00001E111E10100000070907010118
:1003400000000B0C08080800000E100E011E04042B
:100350001F040404030000111111130D00001111FA
:10036000110A040000111115150A0000110A040AEF
:1003700011000011110F010E00001F0204081F06DA
:10038000080810080806040404000404040C02020F
:100390000102020C1926000000000000000000000D
:1003A000000000000000000000000000000000004D
:1003B0001818000708080711040015000411150A91
:1003C000150A150A150000000000000000000000DA
:1003D0000000000000000000000006091C081C09C5
:1003E0000600000000000000000000000000000007
:1003F00000000000000000000000000000000000FD
:1004000000000000000000000000000000000000EC
:1004100000000000000000000000000000000000DC
:1004200000000000000000000000000000000000CC
:1004300000000000000000000000000000000000BC
:1004400000000000000000000000000000000000AC
:10045000001F0404111B1511000000000000000023
:10046000000000000000000000000000000000008C
:10047000000000000000000000000000000000007C
:10048000000000000000000000000000000000006C
:10049000000000000000000000000000000000005C
:1004A000000000000000000000000000000000004C
:1004B000000000000000000000000A1F101C1C10BB
:1004C0001F0E11151915110E0E11101C10110E0012
:1004D000000000000000000000000000000000001C
:1004E000000000000E111D1B1D1B0E0A001F04043E
:1004F000041F0000000000000004041F0404001F8B
:100500000E04040404040E04000C0404040E000091
:1005100000000000000000000000000000000000DB
:10052000000006000000000000000A000E111F106D
:100530000E1313121A16121200000E111C110E00C7
:1005400000000000000000000000000000000000AB
:1005500000000000000000000000000A000C04047D
:10056000040E0709111F1111111E10101E11111E6A
:100570001E11111E11111E1F111010101010060A4D
:100580000A0A0A1F111F10101E10101F1515150E34
:100590001515150E11010601110E11111113151962
:1005A0001115111113151911111214181412110724
:1005B000090909090911111B151111111111111145
:1005C0001F1111110E11111111110E1F1111111105
:1005D00011111E1111111E10100E11101010110EFC
:1005E0001F1504040404041111110F01110E0E153E
:1005F00015150E040411110A040A11111212121217
:10060000121F01111111110F0101151515151515E5
:100610001F15151515151F0118080E0909090E11CA
:1006200011191515151910101E1111111E0E110199
:100630000701110E1215151D1515120F11110F05B9
:10064000091100000E010F110F0F08040E11110EF9
:100650000C12141E11110E00001E12101010000EAC
:10066000010F11110E00000E111F100E00001515C4
:100670000E151500000E1106110E000011131519AC
:100680001100041113151911000011121C12110090
:100690000007090909190000111B151111000011AB
:1006A000111F111100000E1111110E00001F111168
:1006B000111100001E11111E1000000E1110110E5C
:1006C00000001F04040404000011110F011E0000AB
:1006D0000E15150E040000110A040A110000121272
:1006E000121F01000011110F010100001515151551
:1006F0001F00001515151F01000018080E090E0037
:10070000001119151519000010101E111E00000E01
:100710001107110E000012151D151200000F110F08
:1007200005192020202020202020202020202020EB
:1007300020202020202020202020202020202020B9
:100740002020202122232425262728292A2B2C2D4E
:100750002E2F4F3132333435363738393A3B3C3D22
:100760003E3F404142434445464748494A4B4C4D31
:100770004E4F505152535455565758595A5B2F5D4E
:100780005E5F606162636465666768696A6B6C6D11
:100790006E6F707172737475767778797A28D12953
:1007A000E97F060704FFFF85868702898A8B8C8D87
:1007B0008E8F902727CBCA95969798019A9B9C9DE0
:1007C0009E9FA0A1A2A3A4A5A6A7A2A9AAABACADD7
:1007D000AEAFB003B2B3B4B5B6B7B54EBABBBCBDDD
:1007E000BEBF41A042A1E045A3A4A5A64BA74D488A
:1007F0004FA8504354A9AA58E1ABACE2ADAE05AF47
:10080000B0B161B2B3B4E365B6B7B8B9BABBBCBDF9
:100810006FBE7063BF79E478E5C0C1E6C2C3C4C5EA
:10082000C6C7868F98A1AA0000000000858E97A0F9
:10083000A90000000000838C959EA70B3331320085
:10084000848D969FA81B3937380F879099A2AB11DA
:100850000403011088919AA3AC141A090615808923
:10086000929BA413050C0712818A939CA50D363424
:100870003508828B949DA60002301900B3BCC5CE0A
:10088000D70000000000B2BBC4CDD60000000000BD
:10089000B0B9C2CBD40B33313200B1BAC3CCD51B03
:1008A0003937380FB4BDC6CFD81104030110B5BE17
:1008B000C7D0D9141A090615ADB6BFC8D113050C97
:1008C0000712AEB7C0C9D20D36343508AFB8C1CAA9
:1008D000D3000230190098A1C5CED7000000000057
:1008E00097A0C4CDD60000000000959EC2CBD40BCB
:1008F00033313200969FC3CCD51B3937380F99A2BC
:10090000C6CFD811040301109AA3C7D0D9141A096D
:100910000615929BBFC8D113050C0712939CC0C942
:10092000D20D36343508949DC1CAD3000230190067
:100930006770793A7B0000000000666F782D3D00FB
:1009400000000000646D765F400B33313200656E4D
:1009500077222A1B3937380F68717A3C7D110403DE
:10096000011069725B3E20141A090615616A73B1A1
:100970003F13050C0712626B745D2F0D363435087A
:10098000636C755EB900023019004750593B28006E
:1009900000000000464F582B260000000000444D88
:1009A000565F240B33313200454E5722251B393711
:1009B000380F48515A2C29110403011049525B2E5B
:1009C00020141A090615414A53822113050C0712F7
:1009D000424B545D220D36343508434C555E23009E
:1009E00002301900E6EFF83A7B0000000000E5EE67
:1009F000F72D3D0000000000E3ECF5FE400B333125
:100A00003200E4EDF6FF2A1B3937380FE7F0F93CE6
:100A10007D1104030110E8F1FA3E20141A090615AD
:100A2000E0E9F2FB3F13050C0712E1EAF3FC2F0D9E
:100A300036343508E2EBF4FDB90002301900C6CFB8
:100A4000D83B280000000000C5CED72B26000000B0
:100A50000000C3CCD5DE240B33313200C4CDD6DF49
:100A6000251B3937380FC7D0D92C291104030110A1
:100A7000C8D1DA2E20141A090615C0C9D2DB2113F9
:100A8000050C0712C1CAD3DC220D36343508C2CB9F
:100A9000D4DD230002301900CEE1F0E0F2E8F2E507
:100AA000F1FC20EA20EEF42EE4E8EBE5F0F36874C4
:100AB00074703A5C5C7368747269682D6D2E636F34
:100AC0006D2E75618813A00FAC0DB80BC409D0074B
:100AD000DC05E803F401FA00205348545249482D3C
:100AE0005052494E5420444953504C415920534D83
:100AF0003830372E33312020762E312E3620525585
:100B000053204431534D3830372E33312020762E48
:100B1000312E36205255532044320B0B0B0B0B0B4E
:100B20000B0B0A0A0A0A0A0A0A0A09090909090929
:100B300080402010080402018040201008040201B7
:100B400080402010080400000000000000000101A7
:100B50000101010101010202020202020102040874
:100B60001020408001020408102040800102040887
:100B700010207501EA0000000091EA0008950FEFCF
:100B80000ABB04E10BBB00E407BB0FE008BB01E0BC
:100B900004BB0FEF05BB01BB02BB07E006B907B9F9
:100BA0009F9905C001E00093EA0024D809C008E13C
:100BB00001BD05E001BD02E00093EA0056D279D301
:100BC00003D0AED67894089500E002BBA8987BD1FC
:100BD00001E0068B00EC14ED21E030E0008311838E
:100BE0002283338332BF0DE701BF0BE003BF09B798
:100BF000016009BF3687089509B70E7F09BF00E07D
:100C000002BBA898089530E0222339F000FD05C00A
:100C10001695079533953217C8F3032F0895BA93A5
:100C2000AA938A93FA93EA933A922A921A920A9290
:100C30007A936A935A934A933A932A931A930A930C
:100C40008FB7ABEEB0E00D911D912D913C911397B4
:100C5000012B022B032B49F00D9112960ED120404F
:100C600030403C932E931E930E93FD010481158119
:100C7000012B39F0048101D104831583012B09F480
:100C800096D6FD0106811781012B41F00681F5D032
:100C900006831783012B11F400E0048B0085118576
:100CA000012B59F408EE13E00087118701E0168547
:100CB00010271687012FB9D204C00085DED0008727
:100CC0001187FD0102851385012B21F00285D5D006
:100CD0000287138707850023A9F00489002391F474
:100CE00000E007870589033019F4C2D00CE109C080
:100CF000043019F4BDD00DE104C0023019F4B8D0AD
:100D00000EE1048B0089005049F00A9561F10A95C3
:100D100009F442C00A9509F475C027C0B1D006890C
:100D2000A1F4002309F087C0979904C00FEF02BB1C
:100D3000A89881C0A89904C00EEF02BBA89A7BC0F6
:100D400002B3000F016002BB76C0002331F00EEF4A
:100D500002BBA89A00E0068B6EC000890395008B49
:100D60000AE0018B68C08CD019F400E0008B63C0EE
:100D70007AD009F060C02AE046B34F7088D0042BC7
:100D80006DD0028B29E002B310E0A89911E066D083
:100D9000038B00890395EACF6BD0238930E00AE00A
:100DA000029F228940917A0146FD0DC043FF08C091
:100DB00047FF03C0E6EDF8E017C0ECE7F8E014C029
:100DC000E2E2F8E011C045FD08C043FF03C0EEE3D6
:100DD000FAE00AC0E4EEF9E007C043FF03C0EAE826
:100DE000F9E002C0E0E3F9E0E00DF11DE20FF31FCE
:100DF0000491FD01048B0489058B348735870AEF44
:100E0000018BC7CF3DD079F42ED0A9F400E0008B40
:100E1000048515850D3D154010F001E0078701E0C0
:100E2000068B00E084CF0AEF018B048515850F5FE8
:100E30001F4F048715878FBF099119912991399107
:100E40004991599169917991099019902990399016
:100E5000E991F9918991A991B99118950095109509
:100E6000D2DEFD01089501890A95018B00230895C2
:100E700000ED17E006831783089501501040089590
:100E800026B32F7004D0022B0F3F1340089503B3F5
:100E900010E00E77000F000F111F000F111F0895B3
:100EA00004EF11E010D004831583089500E00BD007
:100EB00004830583089507D000E006830783048B2D
:100EC00008952FB7F894EBEEF0E00895FADF02856D
:100ED0001385012B11F001E001C000E02FBF089540
:100EE000F0DF028713872FBF0895EDDF00811181A6
:100EF00022813381012B022B032B11F001E0089595
:100F000000E008950A5E1F4F20E005C00F5F1F4FED
:100F10002395223190F4F80130813433B9F73181CF
:100F20003E32A1F73281353389F72381233D29F4FD
:100F300004810A3C11F401E0089500E0089501E005
:100F4000009302010895009102010895BA93AA93B3
:100F5000D80100910201002351F0C7DF002339F4CA
:100F6000E8E9FAE007D0EEEAFAE004D045DEA9911C
:100F7000B991089506E115911D930A95E1F7089539
:100F80000A5E1F4F30E0F80120812A3A21F401E087
:100F9000009303010BC02A3BD1F32F3AC1F33196E2
:100FA0008F012F3BA1F33395363168F30091030194
:100FB0000895BA93AA9320910301222339F0E8E916
:100FC000FAE007D0EEEAFAE004D016DEA991B99172
:100FD000089526E13591D8013D938D012A95D1F7E9
:100FE00008951FB7F894E3E0F1E00081002361F475
:100FF0001ED00F3F19F400E017D014C018D00530F0
:1010000088F001E000830EC00181002359F40FD065
:101010000F3F41F00CD0053028F409D0039504D0DF
:1010200001E001831FBF089540E050E087C740E022
:1010300050E078C7399803C039980EC0399A0FD05C
:101040000000000000000000389800D00AEC0A956B
:10105000F1F700C00895399A02D0389808953A9867
:10106000389A0BBB000000000895A9D001E09BD086
:1010700001D0E4CF06E097D00CE095D008E483D00F
:1010800009E48DD00AE48BD00BE486D00CE4D2DFE7
:101090000BE1D4DF0DE4CEDF05E1D0DF0EE47CD040
:1010A0000FE48AD000E575D001E570D002E568D084
:1010B00003E563D004E564D005E568D006E569D0B2
:1010C00007E57AD008E56BD009E569D00AE55BD081
:1010D0000BE565D00CE563D00DE56ED00EE553D081
:1010E0000FE56AD000E646D001E644D002E651D0D2
:1010F00003E64CD004E641D005E648D006E649D0E8
:1011000007E65AD008E633D009E631D00AE62CD0FB
:101110000BE642D00CE640D00DE63ED00EE624D0E1
:101120000FE64AD000E748D001E746D002E744D0B6
:1011300003E742D004E740D005E73ED006E73CD0C5
:1011400007E73AD008E738D009E736D00AE734D0C5
:101150000BE732D00CE730D00DE72ED00EE72CD0C5
:101160000FE768DF00E0089565DF0EE167CF62DF1B
:1011700000E164CF5FDF08E161CF5CDF08E05ECFB4
:1011800059DF0CE15BCF56DF0FE158CF53DF09E0A9
:1011900055CF50DF06E052CF4DDF01E14FCF4ADFA0
:1011A00004E04CCF08E346DF0FE11EE4015010409D
:1011B000E9F700C0000008953DDF00E03FCF0FEFEA
:1011C00019EF000001501040E1F700C000C0EADF55
:1011D00008E330DF07E512E001501040E9F700C0F6
:1011E000000008E327DF0FE113E001501040E9F7AA
:1011F00000C00000D7DF08E0D6CFAD01E1E3F1E0A9
:1012000024892160248BDF0107C0AD0166D02489C9
:101210002260248BA8E3B1E027E0F80131918F012F
:101220003D932A95D1F7DA0108950093440108957A
:10123000BA93AA939A93382E2FB6F894B801842FB4
:10124000A1E3B1E0FD010589002311F000E02BC00E
:1012500005E011E09CE242E257E0FB010190BF0192
:101260001124400D511DFA014491F80141938F0161
:101270009A9589F78D01025F1F4F43E0F901519163
:101280009F01F80151938F014A95C1F7882311F00E
:101290008D3218F0FD01118A05C001E0FD01018BBE
:1012A0008A95828B01E02FBE832D9991A991B991E6
:1012B0000895B1D108EC19BD08BD1FBD03E00EBDF6
:1012C00000C009B7006209BF089507D0008D002350
:1012D00019F000E0008FF5DF0895E1E3F1E00895F3
:1012E0002497402FFADF0685088307850983008944
:1012F0000A83088119812A813B8155E0459F402D51
:1013000021D6202F2F7100E024FB0EF401E023FBF7
:101310000EF4026022FB0EF4046021FB0EF4086060
:1013200020FB0EF4006124960895BA93AA938A9341
:10133000FA93EA933A922A921A920A927A936A93C9
:101340005A934A933A932A931A930A938FB763D185
:10135000A1E3B1E0FD010189002351F003890023DD
:1013600039F00FE5228930E0F901EB5FFE4F008391
:10137000FD01078925E031E0200F311F168910504B
:10138000A1F01A9549F11A95C9F11A9509F442C0CC
:101390001A9509F484C01A9509F495C01A9509F4B0
:1013A000D9C01A9509F413C120C111E0158B00238F
:1013B00019F400E841DE05C021503040F9010081F8
:1013C0004ADE36D108F414C100E0078B0689039584
:1013D000068B00E0058B0CC111E0158B002319F47E
:1013E00000EC2ADE03C0F901058935DE21D108F4BD
:1013F000FFC00AE330DE00E0FD01E7CF002319F46F
:1014000006E91ADE02C000E026DE0DD1023008F443
:10141000EFC0DACF002319F400E40EDE3EC0013045
:1014200031F401E0058B00E05BDF15DE36C00230F1
:1014300011F401E4F2CF033011F401E0F5CF0430F0
:1014400011F402E4EACF053011F402E0EDCF0630EA
:1014500011F403E4E2CF073011F403E0E5CF0830E4
:1014600011F404E4DACF093011F404E0DDCF0A30DE
:1014700021F400E0058B05E4D0CF0B3011F400E03F
:10148000D4CF0C3011F406E4C8CF0D30C1F30E30C8
:1014900011F407E4C2CF0F3091F3C2D0B8CF048962
:1014A00000FF07C00E7F048B06890395068B00E0C2
:1014B0009EC001FF05C00D7F048B06890E5FF6CF2D
:1014C00007E0068B95C0002319F400E7B5DD3CC0AA
:1014D000013011F40C9137C0023011F401E7F6CF5E
:1014E000033011F401812FC0043011F402E7EECF74
:1014F000053011F4028127C0063011F403E7E6CF6E
:10150000073011F403811FC0083011F404E7DECF67
:10151000093011F4048117C00A3011F405E7D6CF61
:101520000B3011F405810FC00C3011F406E7CECF5B
:101530000D3011F4068107C00E3011F407E7C6CF55
:101540000F3011F400E087DD6BD008F451C000E0EB
:10155000078BB6CF002311F408E7B8CF013011F4A0
:101560000781F1CF023011F409E7B0CF033011F455
:101570000085E9CF043011F40AE7A8CF053011F453
:101580000185E1CF063011F40BE7A0CF073011F44D
:101590000285D9CF083011F40CE798CF093011F447
:1015A0000385D1CF0A3011F40DE790CF0B3011F441
:1015B0000485C9CF0C3011F40EE788CF0D3011F43B
:1015C0000585C1CF0E3009F0BBCF0FE77FCF018D6E
:1015D0000395018F053138F000E0018F01E0008FA5
:1015E00009B70F7D09BF00E06CCF00E0068B078BC9
:1015F0008FBF099119912991399149915991699117
:1016000079910990199029903990E991F9918991EE
:10161000A991B991189500E010E00DBD0CBD089599
:1016200002D000310895FD0107890395078B0895C5
:10163000FADF0731089501C0D4DCA89519D075D11F
:101640000FE91FE001501040E9F700C000000BE473
:1016500011E00BD191DA02304091770109D019F4F1
:10166000E7DD33DE01C0D5D2ABD1002329F3FFCFB4
:1016700028E731E00BE411E0089501E000937B01DD
:10168000089501E000937D0100E010E029CC009373
:101690007E010895009382010895009381010895C9
:1016A000BD01D901FA012481222361F41CD020E07C
:1016B00005C030E2FD013193DF012395FA01368147
:1016C0002317B8F32481213049F420E003C030E22D
:1016D0003D93239536812317D0F305D0FA01068177
:1016E0000A5EDB01089526E1F80131918F013D93F7
:1016F0002A95D1F70895AC01F8013081E22FF0E08E
:101700003197E13020E0F20744F0CF01F801218168
:1017100020830F5F1F4F0197C9F7F8013083CA017B
:101720000895BD01AC01822F90E0020F191F0150F6
:101730001040F80120810197813030E093074CF090
:10174000DC01F8013291F80130830150104011970B
:10175000C1F7F8012083CA01DB0108959A938A93A7
:10176000C80180D0013011F0002341F44BE751E073
:1017700023E831E08C0194DF0093DB0173D0023069
:1017800011F0002349F44BE751E02FEA31E046968F
:101790008C0186DF0093DC01899199910895EBE734
:1017A000F1E01381012F0F7039F000E00483012F65
:1017B000017149F000E00FC0012F007F11F001E03E
:1017C000F5CF00E00895012F027211F001E003C08F
:1017D0001474B9F302E005830681073190F707819D
:1017E0000A3078F701E008956ED0D8016FDB00234E
:1017F00091F5CD0137D0013011F0002371F4209123
:10180000DB0100917F01002303E811E011F473DF95
:1018100001C087DFE3E8F1E01FD024D0023011F0EF
:10182000002381F42091DC0100917F0100230FEA65
:1018300011E011F460DF01C074DFDC015696EFEABD
:10184000F1E00AD0E4ECFAE00091820112E0019F9D
:10185000E00DF11D35D03CC006E111911D930A95B4
:10186000E1F708950091800108952DD0C801ABE7FC
:10187000B1E0FD010281002329F000E002830C9316
:1018800001831DC00C910023A9F000E00C9387DFB9
:101890000023A9F08C0162DF04EC1AE0FD0127812E
:1018A00032E0239F000D111DF8010AD001E0FD0177
:1018B000018303C00181002311F08C0195DF08C072
:1018C000059114910DCBBA93AA939A938A93089594
:1018D00089919991A991B9910895BA93AA939A93EC
:1018E0008A9388ED9AE0ABE4B1E00FD08EEE9AE0F7
:1018F00043D9023011F484E09BE0A1E6B1E005D0C9
:1019000089919991A991B991089506E1FC011591E8
:10191000CF011D930A95D1F7089531D9DEDF8BCE23
:101920000FEF0FB900EC0DB908954FD14FB6F894F1
:10193000C801ADEDB1E0FD014381442389F145E1EA
:1019400052E06CE2FA017191AF01F80171938F01DD
:101950006A95C1F701E412E043E0F80151918F016B
:10196000F90151939F014A95C1F7BFDA002349F06D
:10197000EADA002331F405E112E0C4DA002309F0C9
:10198000DEDAE1DA002311F08C01E0DA05E112E0A1
:10199000F7DA002311F08C010CDB00E0FD0103837A
:1019A0004FBE89919991A991B99149900895EDED12
:1019B000F1E000E00083028379DA0FEF0FB90895B8
:1019C0001FB7F894EDEDF1E000810023B9F4048134
:1019D000B69907C0002329F401E0048303E00583DE
:1019E0000DC0002359F0B69B03C000E0048307C07C
:1019F00005810A95058311F401E0F8CF00E01FBFCF
:101A00000895E3D0FA93EA933A922A921A920A92AC
:101A10007A936A935A934A933A932A931A930A931E
:101A20004FB60EB12FB1067091F0C1DF4FBE0991D4
:101A30001991299139914991599169917991099017
:101A4000199029903990E991F991ABDF1895A3EE9F
:101A5000B1E08DED91E0FC01428150E08D01040F79
:101A6000151F3081332339F03A95D9F03A95C1F1F9
:101A70003A9531F1DACF2B3121F401E000830FE206
:101A80000AC02D3121F403E0008308E004C02C31AA
:101A900061F602E0008301830091FF000FB900DAD4
:101AA000C5CF99D0E1F705E112E09D014FE2F901C0
:101AB00051919F0185D0D9F701E0FC010383B5CF97
:101AC0008AD069F70C91002319F00A9529F0ADCF5F
:101AD00011968D0192DBA9CF11968D0196DBA5CFD2
:101AE0007DD0013029F40C910031C9F645D80FB9E9
:101AF000FC010181002399F6FD0101811C911E5D0D
:101B000009F448C01B5009F44AC0115259F01A9503
:101B100089F11A95B1F11A95B1F1125041F11A9566
:101B2000A1F183CF002339F4E5E1F2E00CE244D0E7
:101B300009F47BCFFCCF013039F4E5E1F2E006E1B6
:101B40003BD009F472CFFCCF023039F4EBE2F2E083
:101B500006E132D009F469CFFCCF033009F065CF3C
:101B6000E1E4F2E003E028D009F45FCFFCCF00937A
:101B700077015BCF002311F484DD57CF88DD7DDD55
:101B800054CF8BDD52CF86DD50CF002309F04DCFEF
:101B900092D94BCF0CD009B70F7B09BF46CF07D0E6
:101BA000F89405B7006205BF889578943ECFE4D7D6
:101BB000013009F4D898089510E211930A95089518
:101BC000F80151938F014A9508954A92BA93AA93C6
:101BD0009A938A93089502D00023089531813A950B
:101BE0003183F8012083FC010281039502835FB9F0
:101BF0000181089500E010E00DBD0CBD04EB1BBD9C
:101C00000ABD1FBD0BE00EBD09B7006409BFD89A1D
:101C100008955B2F6A2FD801E5E0F1E00CE21D91F9
:101C200011930A95E1F7AFE3B1E003E0F9011191F7
:101C30009F011D930A95D1F7442311F04D3220F0F6
:101C400000E00093420106C001E0009342014A9582
:101C500040934301A62FB52F0895BA93AA939A9360
:101C60008A93FA93EA933A922A921A920A927A9370
:101C70006A935A934A933A932A931A930A933FB6D4
:101C8000DC9AA4E4B2E020E00AE11BE0FD01428D11
:101C900050E0040F121FF801049110E0FD01E00F65
:101CA000F21F2687DB9AFD01028D0395028F063114
:101CB00008F0228F228D30E0E0E3FBE002D1449176
:101CC000EAE1FBE0FED00491FD01E00FF51F46873D
:101CD000E6E4FBE0F6D00491F801E15CFE4F008100
:101CE000ECE5FBE0EED01491102311F011E001C0FF
:101CF00010E0DB980000DC98FD01028D802F90E061
:101D000045E051E0400F531FFA016081603831F423
:101D100021E331E0D9D0E4D0A9F0FDCF613831F42E
:101D200028E331E0D1D0DCD069F0FDCF22E230E011
:101D3000262E67E0629D200D311DC6D0F901159059
:101D4000D1D0E1F7FA016689603831F421E331E05E
:101D5000B3D0BED0A1F0FDCF613831F428E331E03B
:101D6000ABD0B6D061F0FDCF22E230E047E0469F35
:101D7000200D311DA1D0F9017591ACD0E1F7209172
:101D800042012223F1F0209144012223D1F020E0EE
:101D900030E040914301401709F49D0150E0469620
:101DA0004817590719F49D01295F3F4F022F032B54
:101DB00041F006E0F90151939F010A95D9F70FE12F
:101DC0000083FD0121810C916FD0368B038130E4BB
:101DD000239F328162D0258B0295007F2481269536
:101DE000202B248B0681248120FB20E027F93581DC
:101DF000330F330F322B202F269526952695232B34
:101E0000238B0295007F000F2781202B228B2185B9
:101E100000854AD0318B038530E4239F32853DD045
:101E2000208B0295007F24852695202B278704850B
:101E300000FB00E007F92585220F220F202B2687C3
:101E4000112319F0022F016006871E969D010CE0F8
:101E5000F90141919F0118E0DA9840FB16F4D99AF4
:101E600001C0D998DA9A46951A95B1F70A950023D8
:101E700079F73FBE09911991299139914991599169
:101E8000699179910990199029903990E991F99186
:101E900089919991A991B9911895330F3029202FE3
:101EA00022952F70232B0895000F000F000F322F63
:101EB00036953695302B0895AD01495F5F4F67E049
:101EC0000895E20FF51F0895BD01E7E00E2E089575
:101ED000F90171919F01FA017193AF016A9508951B
:101EE000F90111909F01FB011192BF010A9408951D
:101EF00000008895FECF09EE0DBF00E00EBFC0EADE
:101F0000D0E028D0002309F035D007DDF1DFF0CF95
:101F1000E199FECF08954F5F5F4FFADF4EBB5FBB85
:101F2000E09A0895FADF0DB308954F5F5F4F4EBBFF
:101F30005FBBF894E29AE19A0FBE08950FB6E8DF0E
:101F40000DBBF5CF4A952AF036952795179507953D
:101F5000F9CF089501E0089520E006D0E9F708954B
:101F6000259102D0E9F708952D9301501040202FBC
:101F7000212B089582E79BE0FC0105911491FC015F
:101F80003296A591B491FC01349625913491422F5B
:101F9000432B19F0F901E4DF01C0DEDF06961BE0F8
:081FA0008837910748F308950A
:0400000300000000F9
:00000001FF
